:100000002B2AFF3FFF3FFF3F0D3003138312FB00FE
:10001000FF30FA00FB0B0D281028FA0B0D280A28D8
:10002000F330FA00FA0B1228000000000800063036
:1000300003138312FC00FF30FB00FF30FA00FC0BBF
:1000400022282928FB0B25282828FA0B25282228D6
:100050001F281A30FB00FF30FA00FB0B3028332832
:10006000FA0B30282D284230FA00FA0B3528000010
:10007000080003138312B0030319080000000000F6
:100080000000392808001030031383168500013062
:100090008600013083120605F1007108003A031D45
:1000A0005F280030051A0130F1007108003A031D85
:1000B0005C28F030A0005E28E030A0006B28003003
:1000C000051A0130F1007108003A031D6A28D0308A
:1000D000A0006B28A00108000313831686012030BE
:1000E00083128600042004200420860104200420BA
:1000F00008000313831686018030831286000420D3
:100100000420042086010420042008000313831621
:100110008601A03083128600042086010420080096
:10012000031383168601831286010800013003132E
:100130008312AB0017202B080A3A0319A128AB0A37
:100140009A28080003138312AB0CAB132108840018
:100150000130AE00AF0101302C02031CE028013059
:10016000F2002208F1007208F00071080319BC289F
:10017000F00D7010FF3FB628700880042B08B00007
:1001800039200130F2002208F1007208F0007108F5
:100190000319CE28F00D7010FF3FC828F009700831
:1001A00080052B08B00039202F082D06031DDA2802
:1001B0002C082E060319E028AE0A0319AF0AAB2853
:1001C0000800013003138312A30005140830FA005D
:1001D000FA0BE8280000000005100330FA00FA0BC3
:1001E000EF282308283A0319F728A30AE528063040
:1001F000FA00FA0BF92800000800013003138312FB
:10020000A30005150830FA00FA0B042900000000CD
:1002100005110330FA00FA0B0B292308283A0319B9
:100220001329A30A01290630FA00FA0B1529000048
:100230000800031383122908A10084170130F2007B
:100240002A08F1007208F000710803192B29F00D3B
:100250007010FF3F2529F009700880052A08A200C8
:100260000800013003138312A90017202908043A5B
:1002700003193C29A90A3529080043202008E03A3F
:10028000031D43296C202008D03A031D48297920FA
:100290002008F03A031D4D2986202008003A031D4E
:1002A000682990209620F430AB00C830AC00AD0136
:1002B000A2209620F430AB00C830AC00AD01A220E3
:1002C000A0308600F430AB003230AC00AD01A2208B
:1002D00008000230031383168500E12000308518E2
:1002E0000130F1007108003A031D8529FD2000301E
:1002F00085180130F1007108003A031D8229F030A1
:10030000A4008429D030A4009229FD200030851853
:100310000130F1007108003A031D9129E030A4007A
:100320009229A4010800031383168601A0308312CA
:100330008600042004208601C830AB002830AC00C1
:10034000AD01A2200800E33003138312AB00643038
:10035000AC00AD01A2200800CA3003138312AB0029
:100360006430AC00AD01A2200800BE30031383123C
:10037000AB006430AC00AD01A2200800AA3003132A
:100380008312AB006430AC00AD01A22008009830AD
:1003900003138312AB006430AC00AD01A22008004F
:1003A0008F3003138312AB006430AC00AD01A22088
:1003B00008007F3003138312AB006430AC00AD0142
:1003C000A2200800723003138312AB006430AC002B
:1003D000AD01A2200800653003138312AB00643026
:1003E000AC00AD01A22008005F3003138312AB0004
:1003F0006430AC00AD01A220080055300313831215
:10040000AB006430AC00AD01A22008004C300313F7
:100410008312AB006430AC00AD01A220080047306D
:1004200003138312AB006430AC00AD01A2200800BE
:100430003F3003138312AB006430AC00AD01A22047
:1004400008000313831686015030831286000420AF
:100450008601042008000313831685018601831298
:1004600086010530A9000330AA001921F430AB0041
:100470006430AC00AD01A2201720850107309F0039
:1004800098130313123083168500383081008B01D6
:1004900001308600FF3083128100962096200030C4
:1004A0000B190130F1007108003A031D582ACC2ABB
:1004B0000B110108A500312125080106031DCA2AD8
:1004C000A50A0130A30001302502031C742AF43070
:1004D000AB006430AC00AD01A22017202308250634
:1004E0000319742AA30A632A2508013A031D792AED
:1004F000CC2A2508023A031D7E2AEA2A2508033A57
:10050000031D832A122B2508043A031D882A3F2B3A
:100510002508053A031D8D2ACA2B2508063A031D16
:10052000922AEC2B2508073A031D972A1A2C250836
:10053000083A031D9C2A352C2508093A031DA12AD7
:10054000182D25080A3A031DA62A182D25080B3A4E
:10055000031DAB2A182D25080C3A031DB02A182DAF
:1005600025080D3A031DB52A182D25080E3A031D3E
:10057000BA2A182D25080F3A031DBF2A182D250861
:10058000103A031DC42A182D2508103C0318C92A47
:100590004A2ACC2A1720592A3D2169212408E03A09
:1005A000031DD52A93213D21D52A2408D03A031DC5
:1005B000DC2A93213D21DC2A2408F03A031DE92A94
:1005C0009020F430AB006430AC00AD01A2200420D8
:1005D000CD2ACC2A43202008E03A031DF02A6C20C3
:1005E0002008D03A031DF52A79202008F03A031D8F
:1005F000FA2A86202008003A031D112B9020312171
:10060000F430AB00C830AC00AD01A2204030860011
:100610001720F430AB006430AC00AD01A22086019D
:100620003121EA2A43202008E03A031D182B6C20D0
:100630002008D03A031D1D2B79202008F03A031D15
:10064000222B86202008003A031D3E2B90203121CA
:10065000F430AB00C830AC00AD01A2206921240801
:10066000F03A031D3D2B0130A60086202608323AC1
:1006700003193C2BA60A352B122B222B122BFF30F1
:1006800083168600013083120605F1007108013AD5
:10069000031D8A2B003086180130F1007108003AE2
:1006A000031D532BA321003006190130F1007108FE
:1006B000003A031D5C2BAC21003086190130F1009B
:1006C0007108003A031D652BB5210030061A013070
:1006D000F1007108003A031D6E2BBE210030861A0E
:1006E0000130F1007108003A031D772BC72100305B
:1006F000061B0130F1007108003A031D802BD02148
:100700000030861B0130F1007108003A031D892B6F
:10071000D921C92B003086180130F1007108003A48
:10072000031D932BE221003006190130F1007108FE
:10073000003A031D9C2BEB21003086190130F1009B
:100740007108003A031DA52BF4210030061A013070
:10075000F1007108003A031DAE2BFD210030861A0E
:100760000130F1007108003A031DB72B062200305A
:10077000061B0130F1007108003A031DC02B0F2247
:100780000030861B0130F1007108003A031DC92BAF
:1007900018223F2B1030831685000130860001306F
:1007A00083120605F1007108013A031DDC2B861740
:1007B000061304208613DD2B86130030051A013042
:1007C000F1007108013A031DEA2B86160612042077
:1007D0008612EB2B8612CA2B831605160030831265
:1007E000051A0130F1007108013A031D092C90200F
:1007F000C830AB003230AC00AD01A2200420013083
:10080000A60021222608503A0319082CA60A012C1A
:10081000192C69212408E03A031D0F2C6C202408B0
:10082000D03A031D142C79202408F03A031D192C0A
:100830008620EC2B69212408E03A031D202C792026
:100840002408D03A031D252C6C202408F03A031DFF
:10085000332C0130A60021222608323A0319322C0B
:10086000A60A2B2C342C86201A2C8316861383126E
:100870008617172086131720F730831686008312F9
:1008800086150030061A0130F1007108013A031D87
:100890004A2C5D2C0030861A0130F1007108013AB3
:1008A000031D532C5D2C0030061B0130F100710834
:1008B000013A031D5C2C5D2C352CA7018230FB0016
:1008C000FF30FA00FB0B652C682CFA0B652C622CB0
:1008D0008730FA00FA0B6A2C000000000030061A7C
:1008E0000130F1007108013A031D782C0130A70096
:1008F0000030861A0130F1007108013A031D822C84
:100900000230A7070030061B0130F1007108013AE0
:10091000031D8C2C0430A7070130A60001302702EC
:10092000031C9F2C2B30AB003230AC00AD01A22059
:1009300017202608270603199F2CA60A8E2C103094
:1009400086001720203086001720303086001720C0
:100950004030860017205030860017206030860017
:100960001720703086001720073083168600831208
:1009700086150030061A0130F1007108013A031D96
:10098000C22CD52C0030861A0130F1007108013AD2
:10099000031DCB2CD52C0030061B0130F100710853
:1009A000013A031DD42CD52C9F2CA8018230FB00CA
:1009B000FF30FA00FB0BDD2CE02CFA0BDD2CDA2CDF
:1009C0008730FA00FA0BE22C000000000030061A13
:1009D0000130F1007108013A031DF02C0130A8002C
:1009E0000030861A0130F1007108013A031DFA2C1B
:1009F0000230A8070030061B0130F1007108013AEF
:100A0000031D042D0430A8070130A6000130280280
:100A1000031C172DC830AB009630AC00AD01A220EE
:100A20001720260828060319172DA60A062DD52CEF
:100A3000182DFF3FFF3FFF3FFF3FFF3FFF3FFF3FBF
:02400E00223F4F
:00000001FF
